:020000040000FA
:020000000428D2
:040002000034003492
:0800080022008C018D018E0124
:100010002100F0309900210030308C0021000030A8
:100020008D00210000308E00230010308C00230052
:100030008D0123008E01210020309E0021000D3013
:100040009D0025000C309300200004309C0020000F
:100050009A0120003F309B0025001F3091002000B6
:100060001C1520008B0100302A23A90001302A230F
:10007000AA0004302A23AB0005302A23AC00083044
:100080002A23C00009302A23AD000A302A23AE00FB
:100090000B302A23AF000C302A23B00022008C0141
:1000A0008D018E012000B401F0302A23C400441CCD
:1000B0000E1344180E17F1302A23C400441C8E136B
:1000C00044188E17F2302A23C400441C8D134418A0
:1000D0008D17F3302A23C400441C0D1344180D1748
:1000E0008623A5232000A201A301A401A501A60146
:1000F000A701A001A1018C1A8E288C1A902800302B
:10010000200203197B283830200203189428A10A02
:100110000C30210203199728A0017B280000000061
:1001200000000000A00A7B28A001A1017B28A001FB
:10013000A1018C1AA7288C1AA928003020020319C3
:100140009928383020020318AD28A0019928000012
:10015000000000000000A00A992896019701A00164
:10016000A101A1158C1AC5288C1AC72800302002BD
:100170000319B228383020020318CB28A20D22140C
:10018000A10BC328CF28A001B22800000000000066
:100190000000A00AB228A20D2210A10BC328A001C2
:1001A000A1018C1ADF288C1AE128003020020319E3
:1001B000D128383020020318E528A001702800005B
:1001C000000000000000A00AD128A001A101A11593
:1001D0008C1AFB288C1AFD28003020020319E8280D
:1001E0003830200203180129A30D2314A10BF9288C
:1001F0000529A001E8280000000000000000A00A76
:10020000E828A30D2310A10BF928A001A1018C1A45
:1002100015298C1A172900302002031907293830B4
:10022000200203181B29A001702800000000000014
:100230000000A00A0729A001A101A1158C1A3129EB
:100240008C1A33290030200203191E29383020026D
:1002500003183729A40D2414A10B2F293B29A00131
:100260001E290000000000000000A00A1E29A40DA5
:100270002410A10B2F29A001A1018C1A4B298C1A43
:100280004D290030200203193D293830200203187F
:100290005129A001DD290000000000000000A00A93
:1002A0003D29A001A101A1158C1A67298C1A692981
:1002B00000302002031954293830200203186D2918
:1002C000A50D2514A10B65297129A0015429000051
:1002D000000000000000A00A5429A50D2510A10B64
:1002E0006529A001A1018C1A81298C1A832900306B
:1002F0002002031973293830200203188729A0012E
:10030000DD290000000000000000A00A7329A00100
:10031000A101A1158C1A9D298C1A9F290030200259
:1003200003198A29383020020318A329A60D2614A0
:10033000A10B9B29A729A0018A2900000000000029
:100340000000A00A8A29A60D2610A10B9B29A00156
:10035000A1018C1AB7298C1AB9290030200203197F
:10036000A929383020020318BD29A001DD29000089
:10037000000000000000A00AA929A001A101A11508
:100380008C1AD3298C1AD529003020020319C029D0
:10039000383020020318D929A70D2714A10BD12921
:1003A000DD29A001C0290000000000000000A00A13
:1003B000C029A70D2710A10BD12922082306240646
:1003C000250626062706031D7028A21F342A221B95
:1003D000342A2308FE39A80022082906031DFE2915
:1003E00028082A06031DFE292318FA294214C210E0
:1003F00042157028C21442104215702822082B069C
:10040000031D102A28082C06031D102A23180C2A65
:10041000C2154212C21670284216C211C2167028A6
:1004200022082D06031D222A28082E06031D222A33
:1004300023181E2A4314C31043157028C3144310F5
:100440004315702822082F06031D342A2808300679
:10045000031D342A2318302AC3154312C3167028EB
:100460004316C311C31670282209031D392AB4018B
:10047000702822080319122BA21B4E2A7039703AD9
:100480000319872AB4011C302A23B100B11A70283D
:1004900000302A232206031D7028682AB4011C306C
:1004A0002A23B100B11E70282208193E03187028B3
:1004B00010302A232206031D702811302A23230618
:1004C000031D70282408A3002508A4002608A50001
:1004D0002308E039B700203A031970283708803A1A
:1004E000031970283708E03A031970283708003AD2
:1004F0000319122B3708403A031970283708603A5D
:10050000031970283708A03A031970287028341C82
:10051000422AA5080319CF2A2208783A0319992AF2
:100520002208743A0319B72A22087C3A0319BF2A11
:100530007028241A702823082A23B500AA22B5059A
:10054000A41DA62A3508031D642370283508031945
:100550006423702802308A00240807398207013496
:1005600002340434083410342034403480342308F6
:100570002A232402031D7028B40164237028073045
:100580002306031DC82A08302406031D612B392BBE
:100590002408B60023081923B40164237028221DFF
:1005A000E02AA2187028221CFD2AD62A2308B200AD
:1005B000B2030310B20D0310B20DB41464237028FB
:1005C000B41C7028220803393207B3000730330601
:1005D0000319302BA21DF42A2308B600330819236F
:1005E000B301B4016423702833082A232302031DB6
:1005F0007028B301B40164237028B41C7028A21DB4
:10060000092B2308B6001C301923B201B40164235E
:1006100070281C302A232302031D7028B201B40164
:100620006423702822082306031D70283414200038
:1006300070286400230091002000360823009300F6
:10064000151555309600AA30960095149518262B4E
:100650002000080023009100151413082000080052
:1006600008302306031D612B392B08302506031D96
:1006700070288130B60000301923F830B600013000
:1006800019237D30B600023019238130B6000430C2
:100690001923FA30B60005301923C830B6000830E7
:1006A00019238130B60009301923FC30B6000A3016
:1006B00019238130B6000B301923FE30B6000C3000
:1006C0001923B201341004288D120E140630BD0017
:1006D0000A30BB00A030BC0000000000BC0B6C2B3B
:1006E000BB0B6A2BBD0B682B0E10080002302A23AF
:1006F000BD000A30BB00A030BC0000000000BC0BF5
:100700007D2BBB0B7B2BBD0B792B080021009D148F
:100710009D18882B21001C0820004002031C992BE7
:10072000912B42130000C10AC11EA02B1F30C10033
:10073000A02B421700000C1441080319A02BC10381
:1007400041082500910020000800421F0800421DBA
:10075000CF2B421CBD2B8D1200000C1000000E147C
:1007600000000E1300000030B600F030192376238D
:100770000E1042110000421308000E1000000C1071
:1007800000008D1600000E1700000130B600F0309A
:10079000192376238D124211000042130800C21E55
:1007A000F72BC21DE52B0D1200000C1000008E145B
:1007B00000008E1300000030B600F13019237623BC
:1007C0008E10C2120000421308008E1000000C10A0
:1007D00000000D1600008E1700000130B600F13049
:1007E000192376230D12C212000042130800431D84
:1007F0001F2C431C0D2C0E1100000C1000008E1538
:1008000000008D1300000030B600F230192376236B
:100810008E1143110000421308008E1100000C10CD
:1008200000000E1500008D1700000130B600F230F8
:10083000192376230E114311000042130800C31E32
:100840000800C31D352C0C1100000C1000000E1602
:1008500000000D1300000030B600F330192376239A
:100860000E12C3120000421308000E1200000C10FA
:1008700000000C1500000D1700000130B600F33029
:10088000192376230C11C31200004213080008003C
:020000040001F9
:02000E00A40F3D
:02001000FF3FB0
:10E000008100F8007D0001008100FA000A009C00F8
:0AE01000C8008100FC008100FE0042
:00000001FF
